:100000000C94E3010C94FE010C949F040C947B046B
:100010000C94FE010C9480170C94FE010C94FE01CC
:100020000C94FE010C94FE010C94C3170C94FE0179
:100030000C94FE010C94FE010C94FE010C94FE0144
:100040000C94FE010C94FE010C94FE010C94FE0134
:100050000C94FE010C94FE010C943E051D5A344094
:10006000E17A34406ABC344091ED34407D3F354004
:10007000A47035402DB23540F2D23540B6F335404C
:100080003F353640666636408D97364017D9364044
:10009000643B3740EE7C374014AE37409EEF37402C
:1000A000B0723840E926394021B03A4093183C40BC
:1000B000350060008000B0001D013D015A017A0149
:1000C0009701B901DA01F901160240026D028202BC
:1000D000A202EF023203B003F203AA03A703A403B0
:1000E000A1039E039B039803940391038D038A034A
:1000F000860382037E037B03770372036E036A0326
:10010000660361035D03580353034F034A0345032A
:1001100040033B03360330032B03260320031B035A
:1001200015030F030A030403FE02F802F202EC02B5
:10013000E602DF02D902D302CC02C602BF02B90234
:10014000B202AC02A5029E02970291028A028302C9
:100150007C0275026E02680261025A0253024C026E
:1001600045023E0237023002290222021B0215021A
:100170000E0207020002F901F201EC01E501DE01C5
:10018000D801D101CB01C401BE01B701B101AA015F
:10019000A4019E01980192018C01860180017A01DF
:1001A00074016E01680163015D01580152014D0146
:1001B000470142013D01380133012E01290124018B
:1001C0001F011A01150111010C0108010301FF00B3
:1001D000FB00F600F200EE00EA00E600E200DE00BE
:1001E000DB00D700D300CF00CC00C800C500C200A0
:1001F000BE00BB002F03390342034B0353035C03D0
:1002000064036C0373037B03820388038F039503EA
:100210009B0326031C0312030703FD02F202E702FD
:10022000DC02D002C502B902AD02A1029502890228
:100230007C027002630257024A023E023202250229
:1002400019020C020002F401E801DC01D001C40132
:10025000B801AD01A20196018C01810176016C010A
:10026000620158014E0144013B0132012901200184
:1002700017010F010701FF00F700F000E900E1009E
:10028000DB00D400CD00C700C100BB00510A802AAA
:100290000040000A510A084059551801111E111B4F
:1002A000500B411B411F1101511F511B0000000049
:1002B0000880001A204000000000510F91394114BD
:1002C0009131411E410E411D500F8020101548866E
:1002D0004014780570855115510E5195518E21901D
:1002E00081205015484450C528C028200950411489
:1002F000208011110000001054696D6572320041B8
:1003000055544F00445249004D414E00534554004E
:100310004F5054494F4E004D53544F50004D53547D
:100320004152540041535441525400445249525591
:100330004E0053484F4F54005741495400434F55C6
:100340004E540044205354525400442053544F50B0
:100350000042555A5A4552004F4E004F4646004300
:100360004C49434B004F4E004F4646004C4544001D
:100370004F4646004F4E004C4947485400415554A3
:100380004F0054454D5000000102030405040500D0
:1003900001020304050203000159594D4D44440074
:1003A0004D4D444459590044444D4D59590032343F
:1003B000480031324800313248003234480032348B
:1003C00048003132480011241FBECFEFD4E0DEBF19
:1003D000CDBF12E0A0E0B1E0E2E7F3E302C0059098
:1003E0000D92A631B107D9F712E0A6E1B2E001C043
:1003F0001D92AA39B107E1F70C94EA070C940000AA
:1004000040E050E08B9A839A80917A0080688093D4
:100410007A0080917A00806480937A0080917A00DB
:1004200084FFFCCF30E080917A00806480937A0072
:1004300080917A0084FFFCCF209178008091790030
:100440009927982F8827820F911D480F591F3F5FCA
:10045000383048F38B98839880917A008F77809317
:100460007A00CA0123E0959587952A95E1F70895CA
:1004700080937C0083E880937A000E9400020895B4
:100480009F92AF92BF92CF92DF92EF92FF920F9323
:100490001F93CF93DF93C0E0D0E099240E94000225
:1004A0009C0180917C00882309F09DC0809100010F
:1004B000833009F04CC083E02B3238078CF0AE015A
:1004C000FA01EC50FE4F859194918217930730F416
:1004D00093944E5F5F4F99E1991590F76DE216C0C6
:1004E000E3E020323E078CF4AE01FA01EE5EFD4FF0
:1004F000859194912817390730F493944E5F5F4F9C
:10050000F3E6F91590F76BE201C060E281E00E942A
:100510008C06892D0E94FF039FE0A92EA82220E3CC
:10052000A20E182F12951F70120F60E280E00E9439
:100530008C06612F82E00E948C066A2D83E00E9467
:100540008C066AE284E00E948C0663E447C0843033
:1005500009F049C1E92DFF27EE0FFF1FE652FF4FBB
:10056000859194918217930720F093948DE88915D3
:1005700088F7892D0E941004EC0193E6991560F428
:100580006BE280E00E948C068D2F992787FD9A955B
:10059000182F105D612F05C060E280E00E948C067C
:1005A0006BE281E00E948C060FE0A02EAC22E0E31B
:1005B000AE0E14E0D595C7951A95E1F78C2F8F7084
:1005C0008E0F682F82E00E948C066A2D83E00E94C5
:1005D0008C066AE284E00E948C0666E485E00E9454
:1005E0008C0660E0FDC080917C00813009F0BFC0C6
:1005F000E90182E00E9438020E9400029C0140E072
:1006000050E0FA01E055FF4F8591949182179307CE
:1006100030F493944E5F5F4FF6E1F91590F799200F
:1006200029F486EF98E2A4E3B0E419C025E1291586
:1006300028F48AEB99E4ACE3B0E411C0292D332708
:10064000220F331F220F331F245A3F4FF901E59029
:10065000F490F901329605911491D801C701809365
:10066000010190930201A0930301B0930401A1E062
:100670009A2E90927C00CE01AA2797FDA095BA2FC2
:10068000BC01CD010E9405197B018C018091010103
:1006900090910201A0910301B09104019C01AD0170
:1006A000C801B7010E945A19DC01CB0120E030E0FB
:1006B00040E85AE3BC01CD010E945A19DC01CB018C
:1006C00020E030E040EC50E4BC01CD010E945A191A
:1006D0007B018C010E94E8185B016C01862F992731
:1006E000AA2797FDA095BA2FBC01CD010E9405193C
:1006F000DC01CB019C01AD01C801B7010E94A51826
:10070000DC01CB0120E030E048EC52E4BC01CD013B
:100710000E945A19DC01CB01BC01CD010E94E818EE
:100720007B018C018A2D0E94FF03FFE0AF2EA822DF
:10073000F0E3AF0E8E2D0E94FF03182F12951F704D
:10074000105D60E280E00E948C0660E2892D0E94CC
:100750008C0660E282E00E948C066A2D83E00E9493
:100760008C0666E584E00E948C06612F37CFC0912D
:100770007C00C230C1F5809179000E94FF03809116
:100780007800982F9F70E0E3AE2EA90E29E32A157A
:1007900018F477E3A72EA90E682F62956F70162FB5
:1007A000105D1A3308F0195F61E4892D0E948C06F0
:1007B00064E481E00E948C0663E48C2F0E948C0626
:1007C00080917900805D682F83E00E948C06612F04
:1007D00084E00E948C066A2D85E00E948C06692DBB
:1007E00086E00E948C06DF91CF911F910F91FF90C0
:1007F000EF90DF90CF90BF90AF909F900895282FFB
:1008000080E02A3018F08F5F2A50FBCF992734E020
:10081000880F991F3A95E1F7282B822F9927089581
:1008200020E030E0843620F02F5F3F4F8456FACF2F
:1008300054E0220F331F5A95E1F78A3020F02F5FE2
:100840003F4F8A50FACF44E0220F331F4A95E1F719
:100850009927822B932B0895209A229A239A259ADE
:1008600085B1806D85B91DB88EB18C608EB98CE074
:1008700080936B0080ED80936C0080EC8CBB8DBB13
:100880000E943A1880932F02089523B12095207D6D
:100890008CB180958C70282B822F992786FF02C0FF
:1008A00094E00FC027FF02C095E00BC082FF02C09A
:1008B00093E007C083FF02C092E003C084FF16C02C
:1008C00091E080911802882389F080911602882394
:1008D00059F49093170281E08093160280912402CC
:1008E000882311F00E9487181092180280EC8CBBAC
:1008F0001092260208951F920F920FB60F921124A4
:100900002F933F934F935F936F937F938F939F9317
:10091000AF93BF93EF93FF930E944504FF91EF9134
:10092000BF91AF919F918F917F916F915F914F9107
:100930003F912F910F900FBE0F901F9018951F920F
:100940000F920FB60F9211242F933F934F935F9303
:100950006F937F938F939F93AF93BF93EF93FF9387
:100960000E944504FF91EF91BF91AF919F918F91AC
:100970007F916F915F914F913F912F910F900FBE9B
:100980000F901F901895F89480911602882321F0FB
:100990008091170210921602789499270895F99978
:1009A000FECFF89492BD81BDF89A789480B59927CE
:1009B0000895F999FECFF89492BD81BD60BDFA9A71
:1009C000F99AF999FECF7894089581118FEFE1E3B8
:1009D000F2E093E18193915097FFFCCF089580E07E
:1009E0000E94E5048FE08093E70087EB8093E500A9
:1009F00087E08093E60080EC8093E4008091E4003F
:100A000088608093E40010921E020895E82F20E091
:100A100030E0663090F58A52813558F4E13608F0BE
:100A2000EF7DEA52FF27EE0FFF1FE457FD4F2591A0
:100A30003491862F992780FF02C05FE001C050EFFC
:100A40006695E62FFF27EF5CFD4FBC01617070706B
:100A500043E0922F9F7084E0369527958A95E1F7C1
:100A60006115710511F09295907F80818523892B06
:100A700080833596415047FFECCF08951F920F9227
:100A80000FB60F921124DF92EF92FF920F931F93F4
:100A90002F933F934F935F936F937F938F939F9386
:100AA000AF93BF93CF93EF93FF93DD248091180210
:100AB000882361F480911F028F5F80931F0284302E
:100AC00028F081E080931802D0921F0280912302C7
:100AD000833071F4809120028F5F809320028131F6
:100AE00048F081E0809323028FE08093200202C0CF
:100AF0001092200280910501815080930501909110
:100B00003002992371F0882371F480911D028823AB
:100B100021F481E080931E0206C0815080931D0263
:100B200002C090935E02FF2490911E02913009F062
:100B30006CC080911C02853010F4EF2C01C0E92EAE
:100B4000C0E000E010E080915E02992787FD90955B
:100B5000800F911F97FD17C0FF20A9F480915E02BE
:100B6000992787FD9095F801EB5BFD4FE80FF91F82
:100B70008081DF2C87FF02C091E0D92E8F7721F48E
:100B8000FC2EF39401C080E2DD2029F0EE2019F064
:100B90006C2F80E201C06C2F0E940605CF5F0F5FB3
:100BA0001F4FC63080F2ACEEB0E0E1E3F2E0C3E10B
:100BB00081918D93C150C7FFFBCF80911B028111A2
:100BC00081E08093F40080911A029091F9008823CB
:100BD00011F0916001C09E7F9093F90080911902FD
:100BE0009091EE00882311F0906201C09F7D909358
:100BF000EE0081E0F81611F48AEF03C080915E02E6
:100C00008F5F80935E0210921E02809105018823FF
:100C100019F483E08093050180911C028A3019F455
:100C200010921C0203C08F5F80931C02FF91EF9112
:100C3000CF91BF91AF919F918F917F916F915F9174
:100C40004F913F912F911F910F91FF90EF90DF9067
:100C50000F900FBE0F901F901895FC0180911E02FF
:100C60008823E1F7982F8491882391F0AF01A5E4C0
:100C7000B2E09F01F90184918D939F5F2F5F3F4FF9
:100C80004F5F5F4FFA018491882311F0993190F3FF
:100C9000E92FFF27EB5BFD4F1082973048F081E092
:100CA0008093300210925E0283E080931D0204C0A4
:100CB0001092300210925E0281E080931E0208952D
:100CC000DC01E0911E02EE23E1F79E2F8C91882338
:100CD00059F0FD01A5E4B2E081918D939F5F808181
:100CE000882311F09931C0F3E92FFF27EB5BFD4F0B
:100CF0001082973048F081E08093300210925E02BB
:100D000083E080931D0204C01092300210925E02B4
:100D100081E080931E020895893128F4E82FFF278F
:100D2000EB5BFD4F6083089590E2E5E4F2E088E13B
:100D30009193815087FFFCCF089580931B02089503
:100D400090911E029923E1F76093300290935E0226
:100D500080931E02089510921C0208956150704005
:100D6000804090406F3F2FEF72072FEF82072FEFE9
:100D7000920731F02CE70000215027FFFCCFEECF87
:100D8000089560916B0280E090E00E94D904609128
:100D90005F0281E090E00E94D9046091610282E0EC
:100DA00090E00E94D9046091710283E090E00E947B
:100DB000D9046091790284E090E00E94D9046091A6
:100DC000640285E090E00E94D90460917D0286E093
:100DD00090E00E94D90460916F0287E090E00E9449
:100DE000D9046091670288E090E00E94D904609184
:100DF000800289E090E00E94D904609173028AE049
:100E000090E00E94D904609169028BE090E00E941A
:100E1000D90460917B028FE090E00E94D904609138
:100E2000820280E190E00E94D9040895CF93C0E04F
:100E300080E88093610083E080936100C09370003C
:100E400088E08093B60088EC8093B300C0936E0076
:100E500081E0809381008093B0008091B600282FBC
:100E60003327217030708091B6009927847090707C
:100E7000282B392B232B89F768EE73E080E090E074
:100E80000E94AE064FEF51E0F89446BB47BB10926C
:100E90008500109284001092B200B99BFECF109290
:100EA00081007894B09B03C02FEF3FEF0AC0909170
:100EB000840080918500282F3327322F2227290F85
:100EC000311D88E12B36380724F08091660081506F
:100ED00006C0285E374134F4809166008F5F8093AE
:100EE000660001C0C1E050938100CC2369F2CF912C
:100EF00008950E94160790E89093610083E0809324
:100F0000610090BF87E080937F008FE085B980EF1C
:100F10008EB9259A2D9A0E942C040E9479130E9462
:100F2000AB178CE090E00E9466180E94EF040895D1
:100F3000DF92EF92FF920F931F93162FF42ED22E73
:100F4000682F80E00E948C06612F81E00E948C0651
:100F50006F2D82E00E948C066D2D83E00E948C062E
:100F6000602F84E00E948C066E2D85E00E948C0626
:100F700060E086E00E948C061F910F91FF90EF9039
:100F8000DF900895FC014091DD015091DE019A014E
:100F9000240F351F809121029091220228173907D2
:100FA00024F4109222021092210280912102909149
:100FB0002202841795070CF060E28E2F0E948C06A7
:100FC00080912102909122020196909322028093B7
:100FD00021020895CFEFD4E0DEBFCDBF0E94790794
:100FE000789482E080937C000E9438020E94000284
:100FF0001092660280E090E00E94CF0499279093BF
:101000006C0280936B028F3F910521F410926C0269
:1010100010926B0281E090E00E94CF049927909398
:10102000600280935F028F3F910521F4109260026D
:1010300010925F0282E090E00E94CF049927909383
:101040006202809361028F3F910521F41092620247
:101050001092610283E090E00E94CF049927909360
:101060007202809371028F3F910521F410927202F7
:101070001092710284E090E00E94CF04992790932F
:101080007A02809379028F3F910521F410927A02BF
:101090001092790285E090E00E94CF049927909306
:1010A0006502809364028F3F910521F410926502DE
:1010B0001092640286E090E00E94CF0499279093FA
:1010C0007E0280937D028F3F910521F410927E0273
:1010D00010927D0287E090E00E94CF0499279093C0
:1010E000700280936F028F3F910521F4109270027D
:1010F00010926F0288E090E00E94CF0499279093AD
:101100006802809367028F3F910521F41092680274
:101110001092670289E090E00E94CF049927909393
:101120008102809380028F3F910521F41092810209
:10113000109280028AE090E00E94CF049927909359
:101140007402809373028F3F910521F41092740210
:10115000109273028BE090E00E94CF049927909345
:101160006A02809369028F3F910521F410926A020E
:10117000109269028CE090E00E94CF048093630299
:101180008F3F11F4109263028091630280932402D6
:101190008DE090E00E94CF04992790936E02809397
:1011A0006D028F3F910521F410926E0210926D0234
:1011B0008EE090E00E94CF0480937F028F3F11F475
:1011C00010927F028FE090E00E94CF0499279093C5
:1011D0007C0280937B028F3F910521F410927C0268
:1011E00010927B0280E190E00E94CF0499279093B7
:1011F0008302809382028F3F910549F48091070119
:1012000090910801019790938302809382020E943B
:101210009C180E94C304F82E809126029091270208
:10122000839720F088E180936000FFCF80916D026A
:1012300090916E02009709F42B9A8130910509F480
:101240002B98029781F482E080937C000E94380200
:101250000E94000223E0893E92070CF02B98885DE3
:1012600093400CF42B9A20916D0230916E02233042
:10127000310579F4FF2021F0309385022093840218
:101280008091840290918502892B11F02B9801C0E6
:101290002B9A609166026623B1F488EF92E00E9477
:1012A0002D0674E0F71629F488E2809366020C9408
:1012B000731385E0F81611F00C9473138AE0809391
:1012C00066020C9473136A30F9F460E08FEF92E0D9
:1012D0000E942D0624E0F21629F488E2809366022B
:1012E0000C94731365E0F61629F484E1809366028A
:1012F0000C94731372E0F71611F00C9473138BE0D7
:10130000809366020C9473136431F9F460E084E016
:1013100093E00E942D0684E0F81629F48AE0809379
:1013200066020C94731325E0F21629F48EE1809383
:1013300066020C94731362E0F61611F00C947313AA
:1013400085E1809366020C9473136E31F9F460E0CA
:1013500088E093E00E942D0674E0F71629F484E1FA
:10136000809366020C94731385E0F81629F484E6E2
:10137000809366020C94731322E0F21611F00C9421
:10138000731380E2809366020C9473136436F9F44D
:1013900060E08CE093E00E942D0664E0F61629F4EC
:1013A0008EE1809366020C94731375E0F71629F4AE
:1013B00088E2809366020C94731382E0F81611F0B1
:1013C0000C9473138EE6809366020C947313683248
:1013D00031F560E080E193E00E942D0624E0F216F2
:1013E00029F484E6809366020C94731365E0F61684
:1013F00029F48AE0809366020C94731372E0F71666
:1014000029F489E2809366020C94731381E0F81644
:1014100011F00C94731388E180936000FFCF603269
:10142000C1F460E087E193E00E942D062A9A23E050
:10143000F21629F48EE1809366020C94731361E036
:10144000F61611F00C9473138FE1809366020C94DE
:1014500073136F31C9F460E08DE193E00E942D06B3
:101460002A9873E0F71631F42A9A8EE18093660287
:101470000C94731381E0F81611F00C94731380E24E
:10148000809366020C9473136B3009F091C060E096
:1014900084E293E00E942D0623E0F21629F48AE00C
:1014A000809366020C94731361E0F61611F00C94AD
:1014B00073138CE0809366022091690230916A0276
:1014C00088EE93E0289FA001299F500D389F500D72
:1014D0001124209173023091740284E690E0289FD9
:1014E000B001299F700D389F700D1124460F571FB2
:1014F0002091800230918102C90113E0880F991F69
:101500001A95E1F7820F931F820F931F480F591FFF
:101510008091670290916802480F591FCA01AA275B
:1015200097FDA095BA2F8093750290937602A093B1
:101530007702B093780280915F0290916002AC01D3
:10154000C3E0440F551FCA95E1F7480F591F480FD4
:10155000591F2091710230917202C901B3E0880FC6
:10156000991FBA95E1F7820F931F820F931F209165
:10157000610230916202280F391F8CE390E0289FAE
:10158000B001299F700D389F700D1124460F571F11
:1015900080916B0290916C02480F591F4F5F5F4F13
:1015A00050938802409387020E94AB170C947313E8
:1015B0006C3009F0B3C02A9881E00E949D06109219
:1015C0002702109226022091870230918802233050
:1015D000310559F4309385022093840280917F0273
:1015E000882319F081EC809380002230310519F4B2
:1015F000109280005CC0232B09F059C080917502C5
:1016000090917602A0917702B09178020197A1099A
:10161000B1098093750290937602A0937702B093FC
:1016200078020097A105B10541F42A9A8BE08093D6
:10163000660280E00E949D063AC08DE080936602BB
:101640008091640290916502AC01A3E0440F551FA4
:10165000AA95E1F7480F591F480F591F20916F02B3
:1016600030917002C901F3E0880F991FFA95E1F7F4
:10167000820F931F820F931F20917D0230917E0273
:10168000280F391F8CE390E0289FB001299F700D2F
:10169000389F700D1124460F571F80917902909149
:1016A0007A02480F591F5093880240938702209175
:1016B000870230918802C9016CE370E00E94A5198D
:1016C000FB01C9016CE370E00E94A5196C018E2F2B
:1016D0000E94FF03C82F182F1F70105DC295CF7096
:1016E000C05D8C2D0E94FF03982F9F70905D8295A6
:1016F0008F70805DE92E082F212F4C2F60E283E54B
:101700000E94980773E0F71609F0EDC72A9A8BE05C
:101710008093660280E00E949D06E5C76D3009F067
:1017200087C02A9A1092270210922602809187027F
:1017300090918802892BF1F58CE08093660280916C
:101740005F0290916002AC01E3E0440F551FEA95FF
:10175000E1F7480F591F480F591F2091710230912E
:101760007202C90173E0880F991F7A95E1F7820F21
:10177000931F820F931F2091610230916202280F04
:10178000391F8CE390E0289FB001299F700D389F8E
:10179000700D1124460F571F80916B0290916C02BF
:1017A000480F591F4F5F5F4F509388024093870245
:1017B0000E94AB17E0918702F0918802E330F105B7
:1017C00021F4F0938502E0938402CF016CE370E092
:1017D0000E94A5199B01CF016CE370E00E94A5193E
:1017E0006C01822F0E94FF03C82F182F1F70105DFD
:1017F000C295CF70C05D8C2D0E94FF03982F9F7003
:10180000905D82958F70805DE92E082F212F4C2FDF
:1018100060E287E50E94980773E0F71609F063C756
:101820002A9A8BE08093660280E00E949D065BC747
:10183000653109F06FC060E08BE293E00E942D06F5
:1018400020917B0230917C028091820290918302F0
:101850008217930764F490932202809321023093BD
:1018600083022093820290937C0280937B022091DA
:101870007B0230917C0230932202209321028091DE
:10188000820290918302821793070CF43FC0E0918B
:101890002102F0912202EE0FFF1FE75BFE4F60E096
:1018A000808191810E946006109227021092260288
:1018B0002A98E0912102F0912202EE0FFF1FEE0F15
:1018C000FF1FE75FFE4F60817181828193810E94DB
:1018D000AE062A9A8091D9019091DA01A091DB019C
:1018E000B091DC01BC01CD010E94AE0680912102C5
:1018F00090912202019690932202809321022091DE
:10190000820230918302281739070CF684E1809314
:101910006602E9C66E3611F560E082E393E00E944C
:101920002D0684E0F81621F48EE880936602DBC66B
:1019300025E0F21621F488E780936602D4C663E0BE
:10194000F61621F484E680936602CDC672E0F7169F
:1019500009F0C9C68FE680936602C5C66F3609F0E6
:101960005BC081E00E949D0684E0F81631F480910E
:101970006B0290916C02019608C025E0F21649F4C2
:1019800080916B0290916C02019790936C0280930E
:101990006B0280916B0290916C020A9724F0109276
:1019A0006C0210926B0280916B0290916C0297FF17
:1019B00006C089E090E090936C0280936B0263E034
:1019C000F61621F480E7809366020BC071E0F716EB
:1019D00041F48EE68093660280E00E949D060E949C
:1019E000C10620915F02205D90916102905D80911F
:1019F0007102805D50E2E52E022F292F482F6E2DB7
:101A000083E50E94980780916B02805D682F85E0D6
:101A100090E00E94C20767C6603709F05EC081E0AF
:101A20000E949D0684E0F81631F480915F02909147
:101A30006002019608C025E0F21649F480915F0229
:101A40009091600201979093600280935F02809171
:101A50005F0290916002069724F01092600210924B
:101A60005F0280915F029091600297FF06C085E05F
:101A700090E09093600280935F0263E0F61611F4A9
:101A800081E704C072E0F71621F48FE680936602C6
:101A90000BC081E0F81641F48EE68093660280E088
:101AA0000E949D060E94C10690916B02905D20915C
:101AB0006102205D80917102805DE92E00E2482F75
:101AC000602F83E50E94980780915F02805D682FF8
:101AD00084E090E00E94C20706C6613709F05FC04B
:101AE00081E00E949D0624E0F21631F480916102AB
:101AF00090916202019608C065E0F61649F4809163
:101B00006102909162020197909362028093610258
:101B100080916102909162020A9724F01092620211
:101B200010926102809161029091620297FF06C05B
:101B300089E090E0909362028093610273E0F7166F
:101B400011F482E704C082E0F81621F480E7809364
:101B500066020BC021E0F21641F48EE68093660225
:101B600080E00E949D060E94C10620916B02205DCC
:101B700080915F02805D90917102905DE22E082F4E
:101B800020E2492F622F83E50E949807809161022D
:101B9000805D682F83E090E00E94C207A4C5623791
:101BA00009F05AC081E00E949D0664E0F61631F407
:101BB0008091710290917202019608C075E0F7164B
:101BC00049F4809171029091720201979093720290
:101BD0008093710280917102909172020A9724F0B1
:101BE00010927202109271028091710290917202B1
:101BF00097FF06C089E090E0909372028093710293
:101C000082E0F81621F481E7809366020BC021E0A0
:101C1000F21641F48EE68093660280E00E949D06F3
:101C20000E94C10620916B02205D90915F02905D41
:101C300080916102805DE22E092F282F40E2642FFF
:101C400083E50E94980780917102805D682F82E091
:101C500090E00E94C20747C5683711F560E088E34D
:101C600093E00E942D0664E0F61621F48EE6809340
:101C7000660239C575E0F71621F482E880936602A2
:101C800032C583E0F81621F484E6809366022BC502
:101C900022E0F21609F027C589E78093660223C582
:101CA000693709F05BC081E00E949D0664E0F6168A
:101CB00031F48091790290917A02019608C075E022
:101CC000F71649F48091790290917A0201979093E6
:101CD0007A02809379028091790290917A020A9730
:101CE00024F010927A0210927902809179029091F8
:101CF0007A0297FF06C089E090E090937A02809381
:101D0000790283E0F81621F48AE7809366020BC01B
:101D100021E0F21641F488E78093660280E00E9499
:101D20009D060E94C10620916402205D90917D0273
:101D3000905D80916F02805D40E2E42E022F292F9A
:101D4000482F6E2D87E50E94980780917902805D6B
:101D5000682F85E090E00E94C207C5C46A3709F089
:101D60005EC081E00E949D0664E0F61631F4809129
:101D7000640290916502019608C075E0F71649F477
:101D8000809164029091650201979093650280931F
:101D900064028091640290916502069724F010928B
:101DA000650210926402809164029091650297FF2F
:101DB00006C085E090E0909365028093640283E022
:101DC000F81611F48BE704C022E0F21621F489E73B
:101DD000809366020BC061E0F61641F488E78093B9
:101DE000660280E00E949D060E94C10690917902E1
:101DF000905D20917D02205D80916F02805DE92ED3
:101E000000E2482F602F87E50E94980780916402C6
:101E1000805D682F84E090E00E94C20764C46B3745
:101E200009F05FC081E00E949D0674E0F71631F46E
:101E300080917D0290917E02019608C085E0F8169F
:101E400049F480917D0290917E02019790937E02E9
:101E500080937D0280917D0290917E020A9724F00A
:101E600010927E0210927D0280917D0290917E02FE
:101E700097FF06C089E090E090937E0280937D02F8
:101E800023E0F21611F48CE704C062E0F61621F4A8
:101E90008AE7809366020BC071E0F71641F488E789
:101EA0008093660280E00E949D060E94C1062091F8
:101EB0007902205D80916402805D90916F02905D57
:101EC000E22E082F20E2492F622F87E50E94980713
:101ED00080917D02805D682F83E090E00E94C207C0
:101EE00002C46C3709F05AC081E00E949D0684E06C
:101EF000F81631F480916F0290917002019608C03B
:101F000025E0F21649F480916F02909170020197DA
:101F10009093700280936F0280916F029091700293
:101F20000A9724F01092700210926F0280916F0253
:101F30009091700297FF06C089E090E09093700244
:101F400080936F0262E0F61621F48BE780936602BD
:101F50000BC071E0F71641F488E78093660280E0D9
:101F60000E949D060E94C10620917902205D9091F9
:101F70006402905D80917D02805DE22E092F282F02
:101F800040E2642F87E50E94980780916F02805D90
:101F9000682F82E090E00E94C207A5C3623811F565
:101FA00060E08DE393E00E942D0684E0F81621F4B2
:101FB00088E78093660297C325E0F21621F48CE847
:101FC0008093660290C363E0F61621F484E6809362
:101FD000660289C372E0F71609F085C383E880932F
:101FE000660281C3633809F055C084E0F81631F405
:101FF0008091670290916802019608C025E0F21670
:1020000049F4809167029091680201979093680269
:102010008093670280916702909168020A9724F08A
:102020001092680210926702809167029091680294
:1020300097FF06C089E090E0909368028093670262
:1020400063E0F61621F484E88093660208C071E02C
:10205000F71629F482E8809366020E94C106209157
:102060008002205D90917302905D80916902805D95
:1020700030E2E32E022F292F482F6E2D83E40E9499
:10208000980780916702805D682F85E090E00E944C
:10209000C20729C3643809F058C084E0F81631F447
:1020A0008091800290918102019608C025E0F2168D
:1020B00049F480918002909181020197909381026E
:1020C0008093800280918002909181020A9724F08F
:1020D0001092810210928002809180029091810280
:1020E00097FF06C089E090E0909381028093800280
:1020F00062E0F61611F483E804C073E0F71621F4E9
:1021000085E88093660208C081E0F81629F482E829
:10211000809366020E94C10690916702905D2091B3
:102120007302205D80916902805DE92E00E2482FF4
:10213000602F83E40E94980780918002805D682F61
:1021400084E090E00E94C207CEC2653809F059C011
:1021500024E0F21631F4809173029091740201969A
:1021600008C065E0F61649F48091730290917402FC
:1021700001979093740280937302809173029091FF
:1021800074020A9724F010927402109273028091E4
:1021900073029091740297FF06C089E090E09093DB
:1021A00074028093730272E0F71611F484E804C09D
:1021B00083E0F81621F486E88093660208C021E0E7
:1021C000F21629F482E8809366020E94C1062091EB
:1021D0006702205D80918002805D90916902905D30
:1021E000E22E082F20E2492F622F83E40E949807F5
:1021F00080917302805D682F83E090E00E94C207A7
:1022000072C2663809F054C064E0F61631F4809169
:10221000690290916A02019608C075E0F71649F4C8
:102220008091690290916A02019790936A0280936B
:1022300069028091690290916A020A9724F01092D3
:102240006A02109269028091690290916A0297FF76
:1022500006C089E090E090936A028093690282E070
:10226000F81621F485E88093660208C021E0F21692
:1022700029F482E8809366020E94C10620916702D9
:10228000205D90918002905D80917302805DE22ECE
:10229000092F282F40E2642F83E40E949807809141
:1022A0006902805D682F82E090E00E94C2071BC235
:1022B0006C3811F560E083E493E00E942D0664E041
:1022C000F61621F482E8809366020DC275E0F716D7
:1022D00021F48EE88093660206C283E0F81621F4AA
:1022E00084E680936602FFC122E0F21609F0FBC18A
:1022F0008DE880936602F7C16D3809F046C064E04E
:10230000F61631F480917B0290917C02019608C010
:1023100075E0F71649F480917B0290917C02019759
:1023200090937C0280937B0280917B0290917C024F
:1023300020910701309108018217930724F0109231
:102340007C0210927B0280917B0290917C0297FF2D
:1023500006C02150304030937C0220937B0281E004
:10236000F81629F48CE8809366020E94C106E09179
:102370007B02F0917C02EE0FFF1FE75BFE4F60E0F7
:10238000808191810E946006AEC16E3811F560E0D7
:102390008AE493E00E942D0624E0F21621F48CE8F2
:1023A00080936602A0C165E0F61621F48EE6809364
:1023B000660299C173E0F71621F484E68093660201
:1023C00092C182E0F81609F08EC18FE88093660210
:1023D0008AC16F3809F046C024E0F21631F48091CA
:1023E000820290918302019608C065E0F61649F4D6
:1023F000809182029091830201979093830280934F
:102400008202809182029091830220910701309193
:1024100008018217930724F010928302109282021F
:10242000809182029091830297FF06C02150304034
:10243000309383022093820271E0F71629F48EE82C
:10244000809366020E94C106E0918202F0918302AD
:10245000EE0FFF1FE75BFE4F60E0808191810E94DD
:10246000600641C1693211F560E081E593E00E94A8
:102470002D0683E0F81621F488E28093660233C1CA
:1024800022E0F21621F48AE2809366022CC165E014
:10249000F61621F48BE28093660225C174E0F716EC
:1024A00009F021C18FE2809366021DC16A3221F5D5
:1024B00060917F02662321F060E088E593E002C02E
:1024C0008BE593E00E942D0683E0F81649F489E23B
:1024D0008093660260917F028EE090E00E94D904B2
:1024E0002CEFF20E61E06F1508F4FDC080917F02C1
:1024F000862780937F02F7C06B3211F560E08FE58D
:1025000093E00E942D0673E0F71621F488E2809391
:102510006602E9C082E0F81621F48CE2809366023C
:10252000E2C025E0F21621F48DE280936602DBC062
:1025300064E0F61609F0D7C089E280936602D3C042
:102540006C3239F560916302662321F060E085E624
:1025500093E002C088E693E00E942D0673E0F71630
:1025600061F48BE28093660280916302809324027F
:10257000682F8CE090E00E94D9048CEFF80E21E0E7
:102580002F1508F4B0C08091630282278093630204
:10259000AAC06D3211F560E08CE693E00E942D0632
:1025A00063E0F61621F488E2809366029CC072E034
:1025B000F71621F48EE28093660295C085E0F81646
:1025C00021F48FE2809366028EC024E0F21609F0B7
:1025D0008AC08BE28093660286C06E3209F054C0D6
:1025E0002115310521F460E080E793E014C021302B
:1025F000310521F460E084E793E00DC0223031051D
:1026000021F460E087E793E006C02330310529F428
:1026100060E08DE793E00E942D0663E0F61651F42A
:102620008DE28093660260916D028DE090E00E94E1
:10263000D90459C075E0F71689F480916D02909124
:102640006E02019690936E0280936D0204970CF4D3
:102650004AC010926E0210926D0245C084E0F816D6
:1026600009F041C080916D0290916E0201979093A4
:102670006E0280936D0297FF36C083E090E09093E6
:102680006E0280936D022FC06F3209F560E082E820
:1026900093E00E942D0623E0F21621F488E2809355
:1026A000660221C062E0F61621F480E380936602A0
:1026B0001AC075E0F71621F489E28093660213C010
:1026C00084E0F81681F48DE2809366020CC06033DA
:1026D00051F423E0F21619F48FE28093660210920F
:1026E0007C000E94400260E081E00E94A0060C9401
:1026F000090968EE73E080E090E00E94AE06F8946D
:10270000809170008E7F8093700088E08093B60087
:102710001092B2008091B00085608093B0008091EB
:10272000B600282F3327217030708091B60099278A
:1027300084709070282B392B232B89F78FEF87BB60
:10274000809170008160809370007894109288026C
:102750001092870210928D028CE0809386028BE1AA
:102760008093890288E080938C0284E090E09093CB
:102770008B0280938A020895DF92EF92FF920F936B
:102780001F93CF938091EB01882341F480918602BF
:10279000E82FFF27E451FE4F808102C0809186021E
:1027A0000E94FF03C82F2FE0D22ED82280E3D80E3C
:1027B000C295CF70C80F80918D020E94FF03082F31
:1027C0009FE0E92EE82280E3E80E02950F70080FE3
:1027D000809187020E94FF03182F8FE0F82EF122CC
:1027E00080E3F80E12951F70180F6C2F80E00E9486
:1027F0008C066D2D81E00E948C06602F82E00E9485
:102800008C066E2D83E00E948C06612F84E00E946E
:102810008C066F2D85E00E948C0660E086E00E94A9
:102820008C0681E00E949D0660E081E00E94A00687
:1028300080E090E0CF911F910F91FF90EF90DF909B
:102840000895CF92DF92EF92FF920F931F93CF9351
:10285000C82E80911102882361F0809186028093B6
:10286000280280918D0280932902809187028093B3
:102870002A028091EB01882341F480912802E82FFD
:10288000FF27E451FE4F808102C0809128020E9400
:10289000FF03C82F5FE0F52EF82280E3F80EC29503
:1028A000CF70C80F809129020E94FF03182F4FE0BC
:1028B000E42EE82280E3E80E12951F70180F809135
:1028C0002A020E94FF03082F3FE0D32ED82280E384
:1028D000D80E02950F70080F6C2F772780912B026E
:1028E000882309F4606880E00E948C066F2D7727AA
:1028F00080912B02882309F4606881E00E948C0695
:10290000612F772780912B02813009F4606882E083
:102910000E948C066E2D772780912B02813009F45E
:10292000606883E00E948C06602F772780912B02DD
:10293000823009F4606884E00E948C066D2D772750
:1029400080912B02823009F4606885E00E948C0639
:1029500060E086E00E948C0681E00E949D06CC200B
:1029600011F00E94AB0660E081E00E94A00681E0C9
:102970008093110284E0C81649F480912B02E82F5D
:10298000FF27E85DFD4F80818F5F0BC085E0C81693
:1029900051F480912B02E82FFF27E85DFD4F8081E5
:1029A000815080832CC083E0C81641F480912B02B3
:1029B000882311F482E00AC0815008C082E0C81662
:1029C00041F480912B028230C1F08F5F80932B0203
:1029D00016C081E0C81699F4F8948091280280937B
:1029E00086028091290280938D0280912A02992784
:1029F0009093880280938702789410922B028091A2
:102A000028028F3F19F487E18093280280912802E1
:102A1000883110F010922802809129028F3F19F41A
:102A20008BE380932902809129028C3310F010925D
:102A3000290280912A028F3F19F48BE380932A02A6
:102A400080912A028C3310F010922A021092110207
:102A500080E090E0CF911F910F91FF90EF90DF9079
:102A6000CF900895CF93C82F80911202882371F0E0
:102A7000109212026091EB01613019F48EEA93E03A
:102A800003C061E082EB93E00E942D06C43081F424
:102A90006091EB01613029F41092EB0186EB93E039
:102AA00019C081E08093EB01682F8AEB93E012C09C
:102AB000C53099F48091EB01882339F481E080934B
:102AC000EB01682F8EEB93E005C01092EB0161E003
:102AD00082EC93E00E942D0604C0C13011F4C09333
:102AE000120280E090E0CF910895AF92BF92CF9212
:102AF000DF92EF92FF920F931F9380918A020E94C0
:102B0000FF03F82EEFE0CE2EC82280E3C80EF69425
:102B1000F694F694F694F80E80918C020E94FF03CE
:102B2000E82E7FE0B72EB82280E3B80EE694E69454
:102B3000E694E694E80E809189020E94FF03D82E65
:102B40006FE0A62EA82280E3A80ED694D694D69441
:102B5000D694D80E80912502E82FFF270FED11E0C3
:102B6000EE0FFF1FE00FF11F0190F081E02D849127
:102B70006F2D0E948C0680912502E82FFF27EE0F13
:102B8000FF1FE00FF11F0190F081E02D319684913D
:102B90006C2D0E948C0680912502E82FFF27EE0FF6
:102BA000FF1FE00FF11F0190F081E02D329684911C
:102BB0006E2D0E948C0680912502E82FFF27EE0FD4
:102BC000FF1FE00FF11F0190F081E02D33968491FB
:102BD0006B2D0E948C0680912502E82FFF27EE0FB7
:102BE000FF1FE00FF11F0190F081E02D34968491DA
:102BF0006D2D0E948C0680912502E82FFF27EE0F95
:102C0000FF1FE00FF11F0190F081E02D35968491B8
:102C10006A2D0E948C0660E086E00E948C0681E0AE
:102C20000E949D0660E081E00E94A00680E090E0A6
:102C30001F910F91FF90EF90DF90CF90BF90AF90DA
:102C40000895FF920F931F93CF93F82E8091130254
:102C5000882361F080918A0280932C0280918C02FB
:102C600080932D028091890280932E02C0911402DC
:102C7000CC23C9F480912C020E94FF03182F082F47
:102C80000F70005D12951F70105D60E28C2F0E9426
:102C90008C0660E281E00E948C0669E582E00E9479
:102CA0008C0669E535C0C130C9F480912D020E94BF
:102CB000FF03182F082F0F70005D12951F70105D15
:102CC00060E280E00E948C0660E28C2F0E948C06FD
:102CD0006DE482E00E948C066DE41AC0C23019F5E2
:102CE00080912E020E94FF03182F082F0F70005DA5
:102CF00012951F70105D60E280E00E948C0660E219
:102D000081E00E948C0664E48C2F0E948C0664E4AF
:102D100083E00E948C06612F84E00E948C06602F65
:102D200085E00E948C0660E086E00E948C0680E0D0
:102D30000E949D06FF2011F00E94AB0660E081E03A
:102D40000E94A00681E08093130284E0F81649F403
:102D500080911402E82FFF27E45DFD4F80818F5F93
:102D60000BC085E0F81651F480911402E82FFF277C
:102D7000E45DFD4F8081815080832CC083E0F81694
:102D800041F480911402882311F482E00AC081503A
:102D900008C082E0F81641F4809114028230C1F03C
:102DA0008F5F8093140216C081E0F81699F4F894AE
:102DB00080912C02992790938B0280938A028091B4
:102DC0002D0280938C0280912E0280938902789448
:102DD0001092140280912C028F3F19F483E68093A5
:102DE0002C0280912C02843610F010922C028091DB
:102DF0002D02882319F48CE080932D0280912D02FE
:102E00008D3018F081E080932D0280918C02823009
:102E1000C9F420918A0230918B02C90183709070AD
:102E2000892B81F4C90164E670E00E94A519892B01
:102E300039F4C90160E971E00E94A519892B11F4E8
:102E4000EDE107C080912D02E82FFF27EC5FFD4FD9
:102E5000E08180912E02882311F4E0932E0280916C
:102E60002E02E81718F481E080932E0210921302CC
:102E700080E090E0CF911F910F91FF900895CF9344
:102E8000C82F80911502882379F010921502809145
:102E90002502E82FFF27EE0FFF1FEB51FE4F61E0E9
:102EA000808191810E942D06C43049F480912502D1
:102EB000823018F0109225020DC08F5F09C0C53016
:102EC000B9F480912502882311F482E001C0815079
:102ED0008093250280912502E82FFF27EE0FFF1F28
:102EE000EB51FE4F61E0808191810E942D0604C06C
:102EF000C13011F4C093150280E090E0CF910895A5
:102F00001F920F920FB60F9211248F939F9380916F
:102F1000870290918802019790938802809387029C
:102F20008091840290918502009729F001979093F7
:102F30008502809384028091260290912702019657
:102F400090932702809326029F918F910F900FBE3E
:102F50000F901F90189583E0E2E9F2E01192119230
:102F6000815087FFFBCF9FEFEEE8F2E083E0919383
:102F7000815087FFFCCF82E080936E0086E287BDA0
:102F80008CE084BD08951F920F920FB60F9211240A
:102F90000F931F932F933F934F935F936F937F9361
:102FA0008F939F93AF93BF93CF93EF93FF93C3E020
:102FB00002E912E0D801ED91FD918D01309709F001
:102FC0000995C150C7FFF6CFEEE8F2E0C3E080817B
:102FD0008F3F21F0882311F081508083C1503196BA
:102FE000C7FFF5CFFF91EF91CF91BF91AF919F9127
:102FF0008F917F916F915F914F913F912F911F9191
:103000000F910F900FBE0F901F901895AC0120E00C
:10301000E2E9F2E0819191918417950761F02F5FC9
:103020002430C0F320E0E2E9F2E080819181892B35
:1030300029F45183408381E090E008952F5F329618
:10304000243098F380E090E008959C0140E0E2E9AC
:10305000F2E0808191818217930729F41182108216
:1030600081E090E008954F5F3296443090F380E025
:1030700090E0089590E0E92FFF27E257FD4F80810F
:103080009F5F8F3F21F41082892F992708959430F4
:1030900090F380E090E00895F894E82FFF27E3573D
:1030A000FD4F608378940895F894E82FFF27E35745
:1030B000FD4F8081789499270895F894E82FFF2791
:1030C000E357FD4F8FEF8083789408959C01832F01
:1030D00099278093C5002093C40082E08093C000AC
:1030E00080E18093C10086E08093C2000895982F0C
:1030F0008091C00085FFFCCF9093C6000895809119
:10310000C0008823E4F78091C60099270895CF93E3
:10311000C9E02D9A61E070E080E090E00E94AE0688
:103120002D9861E070E080E090E00E94AE06C15012
:10313000C7FFEFCFCF9108951092800089E0809370
:10314000810080E18093880008955058192E84D022
:1031500001D06AC0BA176207730784079507B1F1F7
:1031600088F40EF410940B2EBA2FA02D062E622F89
:10317000202D072E732F302D082E842F402D092E41
:10318000952F502DFF275523B9F0591B49F0573E75
:1031900098F0469537952795A795F0405395C9F730
:1031A00076F0BA0F621F731F841F30F487957795EE
:1031B0006795B795F040939517FA0F2E0895BF1BAA
:1031C000BB27BA0B620B730B840BF6CFDEF670C015
:1031D00097FB4ED09F3738F0FEE9F91B982F872FC9
:1031E000762F6B2F05C061C096958795779567956B
:1031F000F150D0F73EF490958095709561957F4F92
:103200008F4F9F4F0895E89403C097FB0EF4F3DFB0
:10321000B62F672F782F892F9EE9002405C09A9535
:10322000BB0F661F771F881F11249923A1F08823E5
:10323000B2F79F3F59F0BB0F48F421F4002011F47E
:1032400060FF04C06F5F7F4F8F4F9F4F881F979520
:10325000879597F9089529C0052E092607FA440F86
:10326000551F5F3F79F0AA27A51708F051E0479551
:10327000880F991F9F3F31F0BB27B91708F091E0E5
:10328000879508959F919F9111245CC097FB880FAB
:10329000991F9F3F31F0BB27B91708F091E0879540
:1032A00008959F919F9111244DC066277727882705
:1032B00099270895D1DF01D0B7CF992339F055234D
:1032C00029F09F575F57950F13F49AF1F1CF91585A
:1032D0009F3FE1F3629FA12D0F92BB27639FA00D3B
:1032E000B11DEE27729FA00DB11DEE1FAF93AA274F
:1032F000649FB00DE11D739FB00DE11DAA1F6627ED
:10330000829FB00DE11DA61F5527749FE00DA11DE2
:10331000551F839FE00DA11D561F849FA00D511DB9
:10332000852F7A2F6E2F1F900F9088231AF4939574
:1033300039F408C0000C111CBB1F661F771F881FC3
:10334000012808959FEF80EC0895AA1BBB1B51E153
:1033500007C0AA1FBB1FA617B70710F0A61BB70B05
:10336000881F991F5A95A9F780959095BC01CD01AA
:023370000895BE
:10337200039A993940030F10000100000002000077
:1033820000040000000800000010000000210000FE
:1033920000420000007D000000FA000000F401007D
:1033A20000E8030000D0070000A00F0000401F004B
:1033B20000983A000030750000D201CB01C401BD73
:1033C20001B601AF01A801A1019A0193018C018507
:1033D200017E0177017001690120333020207300E2
:1033E2002031352020730020203820207300202037
:1033F200342020730020203220207300202031202E
:10340200207300312F3220202000312F3420202041
:1034120000312F3820202000312F3135202000317B
:103422002F3330202000312F3630202000312F3131
:1034320032352000312F3235302000312F353030F7
:103442002000312F3130303000E8030000010093BA
:10345200038D038703A703A0039903010C01020351
:103462000405060708090A0B0C01020304050607F6
:1034720008090A0B001F1C1F1E1F1E1F1F1E1F1ED6
:063482001F01010102011F
:00000001FF
